:020000040000FA
:100000007C2882070034003400340134003400348A
:1000100000340A34003400340034643400340034D2
:100020000334E8340034003427341034003401340D
:100030008634A03400340F344234403400349834D1
:10004000963480348207123403343634183403343F
:100050003A341C3400343E342134033442348207B1
:100060000A340934083406340534043402340134C3
:1000700082075334773465346534703447346534DB
:100080006E340034203456346534723431342E34B6
:10009000313465340034533474346134723474341C
:1000A000003445346E34643400345334743465346D
:1000B000703400344D34613472346B3465347234CE
:1000C00000345334773465346534703469346E34B5
:1000D00067340034423461346434203445346E343F
:1000E0006434003420344B3448347A34003443349C
:1000F00041344C34203400348B0107309F00980188
:10010000831698018C019F018113FB3085008601C5
:100110008312AD01AE01AF01B001B1018922892284
:100120000515A322C3222930840000309223D10177
:10013000D5010508D00003305005CF00501E2622FF
:100140006F230030B6200330B620D120031CAD2829
:1001500032233130C922BE23A3280630B62009300D
:10016000B6208123DD206F231522A128DA00322357
:100170005A08003E2220C922BE235A08013E2220EE
:10018000D80003010D2232235A08023E2220DD004E
:100190000E2388229B21551ACF282D21CA285512BB
:1001A00008003608AD003708AE003808AF0039083F
:1001B000B0003D30840008210800D5143E30DD0039
:1001C0004C22323020213A300321423003213223A5
:1001D0002830C92205113630DD004C222D30DD00DB
:1001E000E621551A00298922453084000821031888
:1001F000051536213D30840008210318EA28F0282F
:10020000D50105150800DD004C225D0820210800FD
:1002100000083002031C1F29031D1F298403000846
:100220002F02031C1F29031D1F29840300082E020F
:10023000031C1F29031D1F29840300082D02080029
:1002400084002D088000840A2E088000840A2F086C
:100250008000840A300880000800D11831297F21ED
:100260003329362155210E2388220800D7015D0845
:100270008400320880070330D3004F2184038403B5
:10028000330880070230D3004F21840334088007ED
:10029000840A031C4C29800A350880070800570D82
:1002A000840A8007D30B4F29080003305D078400C0
:1002B00002300002031C7E29031D71298403623071
:1002C0000002031C7E29031D712984035A30000299
:1002D000031C7E29031D7129840300300002031CC6
:1002E0007E295D08840000308000840A5A30800036
:1002F000840A62308000840A0230800008008F2166
:10030000362103305D078400801F8D29800184031E
:10031000800184038001840380018F210800B209D9
:10032000B309B409B509B20F9A29B30F9A29B40FCA
:100330009A29B50A0800CA21551AC9290508D0000A
:10034000D32305085006031D9B2903305005CE001A
:100350004F0603199B290310CF0D4E08CF064F08F7
:100360000239D2005106D101CF18BE294E08CF0064
:10037000DC035C189B29DC189B29C7290230D100BB
:100380004E08CF00DC0A5C189B29DC189B294E081C
:10039000CF000800D5180A2A051AE629851DF2297A
:1003A0002030D6005510CA23051AE229851DF229EE
:1003B000D603031DD32901300D220430D600551475
:1003C000D511D3290130D5190A2A052A85190A2AF7
:1003D000CA238519F029D518E829051EF229E8292C
:1003E00055160A2A2030D6005510D515CA23051AED
:1003F000042A8519042AD603031DF629FF300D228D
:100400000430D6005514F629FF3055180A2A0D225B
:10041000051ECA29D5115510080058070739D800FC
:100420002F20D90015220E2308000430D3003530C8
:1004300084005808D7000310D70DD70D57080120A6
:1004400080008403D70AD30B1E2A0800D514363047
:100450008400043092233630DD000E238C304D238F
:100460003E30C92288229B21051A462AB501B401D3
:10047000B3010430D01D8030B200D118402A8F2142
:100480002930DD0036213630DD00322A2930840063
:1004900003019C23D5100800AD01AE01AF01B001EE
:1004A000B1012030D3002908A5002A08A6002B0896
:1004B000A7002C08A8005D0884000310251C7A2AD8
:1004C0000008AE07031C692AAF0F692AB00F692A1A
:1004D000B10A840A0008AF07031C712AB00F712A01
:1004E000B10A840A0008B007031C772AB10A840AFB
:1004F0000008B107B10CB00CAF0CAE0CAD0CA80CE1
:10050000A70CA60CA50C5D08D30B5C2AB101080052
:100510004C222D3084000008C9000830C800C90CE6
:10052000031C962A861506150611992A86110615AA
:100530000611C80B8F2A840A32300402031C8B2A4E
:10054000861786130800C723033086000616C723C4
:100550000612033086000616CA23061203308600F0
:100560000616CA230612023086000616CD2306128E
:1005700020304D2308304D2301304D2306304D23CC
:100580000E304D2308000030C9220930C922BC2397
:100590000800DB003820FF390319D22A5123DB0A77
:1005A0005B08CA2A08002030C600A001A101A201F0
:1005B000A301A4015D0884000008A500840A0008C6
:1005C000A600840A0008A700840A0008A8000310F7
:1005D000A50DA60DA70DA80D03182514A00DA10D9E
:1005E000A20DA30DA40DC603031DF72A0800203099
:1005F00084000323840A0323840A0323840A032335
:10060000840A0323E72A03300007C700C7198000C4
:1006100030300007C700C71B80000800D32202301B
:100620004D2320305123230E2B2323082B232C3042
:100630005123220E2B2322082B23210E2B232E3075
:10064000512321082B23200E2B2320082B23393064
:10065000C9222E2308000F39303E512B8030590417
:100660004D23080001304D23080086018316083011
:100670008600831206138616FF30CC000616060885
:10068000CB00061200000000061600000612CC0384
:1006900003194C2BCB193E2B0800CA00D4010613BA
:1006A000542BCA00541406173523860183160030D4
:1006B000860083128612061354180617F03086053A
:1006C0004A0E0F398604061600000612F030860521
:1006D0004A080F3986040616000006120800363054
:1006E000DD008400083092233A3084000C309223DD
:1006F0003E30840010309223423084001430922324
:1007000008003630840008309C233A3084000C30D6
:100710009C233E30840010309C23423084001430EF
:100720009C230800F0000430D300B5238000F00AB9
:10073000840AD30B952B0800F0000430D300000886
:10074000A623840AF00AD30B9F2B080083169A0075
:1007500070089B001C1555309D00AA309D009C140C
:100760009C18B02B1C1183120800831670089B0084
:100770001C141A0883120800C123C123C123C123FA
:100780000800C423C4230800FF30CC00D52B8030E0
:10079000CC00D52B4030CC00D52B2030CC00D52B35
:1007A0001030CC00D52B0230CC00FF30CD00CD0B6B
:0807B000D72BCC0BD52B080060
:084000005700330043004400A7
:02400E00303F41
:10420000CA0017005C0022008000960098000000A1
:10421000800084001E00000020000B002000000031
:104220006400000000000000D00047001F000000F4
:00000001FF
